:100000000C9432030C9479030C9479030C947903C7
:100010000C9479030C9479030C9479030C94790370
:100020000C9479030C9479030C9406220C94D92235
:100030000C9477190C9479030C9479030C9479033C
:100040000C9479030C9479030C9479030C94790340
:100050000C9479030C94DF190C9479030C947903B4
:100060000C9479030C9479030C9479030C94790320
:100070000C9479030C9479030C9479030C94790310
:100080000C9479030C9479030C9479030C94790300
:100090000C9479030C9479030C9479030C947903F0
:1000A0000C9479030C9479030C94790324002500B3
:1000B0002600250221002200230038001E001F0018
:1000C00020002D002700280037002E00010001002D
:1000D0000100010001000100010001000100010018
:1000E0000100010001000100010001000100010008
:1000F00001000100010001000100010001000100F8
:1001000001000100010001000100010001000100E7
:1001100001000100010001000100010001000100D7
:1001200001000100010001000100010001000100C7
:1001300001000100010001000100010001000100B7
:1001400001000100010001000100010001000100A7
:100150000100010001000100010001000100010097
:100160000100010001000100010001000100010087
:100170000100010001000100010001000100010077
:100180000100010001000100010001000100010067
:100190000100010001000100010001000100010057
:1001A0000100010001000100010001000100010047
:1001B0000100010001000100010001000100010037
:1001C0000100010001000100010001000100010027
:1001D0000100010001000100010001000100010017
:1001E0000100010001000100010001000100010007
:1001F00001000100010001000100010001000100F7
:1002000001000100010001000100010001000100E6
:1002100001000100010001000100010001000100D6
:1002200001000100010001000100010001000100C6
:1002300001000100010001000100010001000100B6
:1002400001000100010001000100010001000100A6
:100250000100010001000100010001000100010096
:100260000100010001000100010001000100010086
:100270000100010001000100010001000100010076
:100280000100010001000100010001000100010066
:100290000100010001000100010001000100010056
:1002A000010001000100010001000100643214643A
:1002B0003214783C1E1E140A0500000000010101E2
:1002C0000202030405050607090A0B0C0E0F1112A2
:1002D000141517191B1D1F212325282A2C2F3134F3
:1002E00036393B3E414346494C4F5255585A5D6161
:1002F00064676A6D707376797C7F8386898C8F9250
:1003000095989B9EA2A5A7AAADB0B3B6B9BCBEC135
:10031000C4C6C9CBCED0D3D5D7DADCDEE0E2E4E682
:10032000E8EAEBEDEEF0F1F3F4F5F6F8F9FAFAFBA2
:10033000FCFDFDFEFEFEFFFFFFFFFFFFFFFEFEFEDA
:10034000FDFDFCFBFAFAF9F8F6F5F4F3F1F0EEED49
:10035000EBEAE8E6E4E2E0DEDCDAD7D5D3D0CECBD8
:10036000C9C6C4C1BEBCB9B6B3B0ADAAA7A5A29E4A
:100370009B9895928F8C898683807C797673706D3B
:100380006A6764615D5A5855524F4C494643413E35
:100390003B393634312F2C2A282523211F1D1B19C8
:1003A00017151412110F0E0C0B0A09070605050488
:1003B0000302020101010000000000000000010131
:1003C0000101010101010102020202020202020214
:1003D00003030303030303030404040404040505E3
:1003E00005050506060606060707070708080808A4
:1003F0000909090A0A0A0A0B0B0B0C0C0C0D0D0D4E
:100400000E0E0F0F0F1010111111121213131414DE
:10041000151516161717181819191A1A1B1C1C1D52
:100420001D1E1F1F202021222223242525262727A9
:1004300028292A2B2B2C2D2E2F2F303132333435D7
:1004400036363738393A3B3C3D3E3F4041424344E3
:10045000464748494A4B4C4D4F50515253555657B9
:10046000585A5B5C5E5F606263646667696A6C6D64
:100470006E707173747678797B7C7E8081838486DC
:10048000888A8B8D8F91929496989A9B9D9FA1A319
:10049000A5A7A9ABADAFB1B3B5B7B9BBBDBFC1C41B
:1004A000C6C8CACCCFD1D3D6D8DADCDFE1E4E6E8DF
:1004B000EBEDF0F2F5F7FAFCFF12036B0065007943
:1004C0000062006F0061007200640000001603719A
:1004D000006D006B006200750069006C00640065CF
:1004E00000720000000403090409026D0004010009
:1004F000A0FA090400000103010100092111010013
:10050000012240000705810308000A0904010001D7
:1005100003010200092111010001224D000705829B
:100520000308000A09040200010300000009211168
:100530000100012236000705830308000A090403AD
:100540000001030000000921110100012239000708
:100550000584032000011201100100000008EDFED7
:10056000606001000102000105010906A101050703
:1005700019E029E715002501950875018102050894
:1005800019012905950575019102950175039101E0
:100590000507190029F71500250195F87501810255
:1005A000C005010980A10185021601002603001A79
:1005B00081002A8300751095018100C0050C090196
:1005C000A1018503160100269C021A01002A9C0243
:1005D000751095018100C005010902A1010901A161
:1005E00000050919012905150025019505750181E9
:1005F0000295017503810105010930093115812535
:100600007F95027508810609381581257F9501754A
:10061000088106050C0A38021581257F95017508A9
:100620008106C0C005010906A101050719E029E7F7
:100630001500250195087501810295017508810154
:1006400005081901290595057501910295017503A4
:1006500091010507190029FF150026FF0095067571
:10066000088100C011241FBECFEFDAE0DEBFCDBF8E
:1006700004B603FE27C080912A0290912B02A0911C
:100680002C02B0912D028730904BA740B04BD1F493
:1006900010922A0210922B0210922C0210922D021C
:1006A00014BE84B7877F84BF0FB6F894A895809155
:1006B0006000886180936000109260000FBEE0E0EF
:1006C000F8E3099511E0A0E0B1E0EEE5FCE402C03A
:1006D00005900D92A033B107D9F722E0A0E3B1E075
:1006E00001C01D92AA32B207E1F70E94531F0C9479
:1006F0002D260C94000090E080E008950895089560
:1007000081E00895089581E008950C9480030E948B
:10071000EC112FEF84E39CE0215080409040E1F702
:1007200000C000000C94041AFF920F931F93CF9304
:10073000DF938C01FC01C081D18180916F01811117
:1007400048C08281882309F43FC0CE010E9451171E
:10075000F82E682FCE010E94F916BE018F2D0E943F
:100760003005EC01B8010E948503882309F478C0A4
:10077000B801CE010E944007882309F471C0C63336
:10078000F0E7DF0709F484C0C0F5C53190E7D90769
:1007900028F5C230E0E7DE0708F099C0C115F0E7A0
:1007A000DF0709F458C0C130D04709F460C081E0C8
:1007B0008093320180933301C801DF91CF911F9163
:1007C0000F91FF900C948303CE010E942717F82EFF
:1007D000C4CFCE010E945117BE01C1CFC43390E7F0
:1007E000D90709F44EC0C533D04709F7F801828113
:1007F0008823B1F10E94180B33C0CA33F0E7DF073A
:1008000009F457C070F4F8018281C833F0E7DF07BC
:1008100009F44AC008F443C0882311F10E945C0A1D
:100820001FC0CC33E0E7DE0709F4D5C008F448C0A8
:10083000CD33D04709F0BBCFF8018281882309F47A
:10084000F1C0109233010E94A91990933101809355
:10085000300180E2CDC0F801828181110E948703BE
:1008600080E0DF91CF911F910F91FF900895F801E3
:1008700082818823A9F38091DF0181608093DF0169
:10088000EFCFF8018281882359F30E94220BE8CF31
:10089000F8018281882321F30E940D0AE1CF882389
:1008A000F9F20E94250ADCCF8823D1F20E94440A83
:1008B000D7CFF8018281882399F20E94740AD0CFA1
:1008C000F8018281882361F20E948C0AC9CFF80165
:1008D0008281882309F470CF0E940919811102C016
:1008E0000E94E8180E94261990E090931C028093C1
:1008F0001B02FE01E350F04780911B028160E23150
:10090000F105C8F4EA57FB4F0C94DF259804A404C2
:10091000A804AC04B004B404B804BC04C004C40407
:10092000C804CC04D004D404D804DC04E004E404F7
:1009300080911B02826080931B0280911B020E94A7
:100940002A190E94EC118CCF80911B028460F3CF96
:1009500080911B028860EFCF80911B028061EBCFFA
:1009600080911B028062E7CF80911B028064E3CFFD
:1009700080911B028068DFCF80911B028460EACFE8
:1009800080911B028E7FD7CF80911B028D7FD3CFAA
:1009900080911B028B7FCFCF80911B02877FCBCFB3
:1009A00080911B028F7EC7CF80911B028F7DC3CFAA
:1009B00080911B028F7BBFCF80911B028F77BBCFB3
:1009C00080911B028B7FEACF90911B02892F97FBAE
:1009D00087F98058B0CFF8018281882361F01092A6
:1009E00032010E94A919909331018093300182E075
:1009F0000E94760F35CF8091320181110FC0809116
:100A00003001909131010E94B519883C910530F474
:100A100086E20E944B0E86E20E94270F82E00E942F
:100A20007D0F1ECF8091330181110FC08091300165
:100A3000909131010E94B519883C910530F487E20C
:100A40000E944B0E87E20E94270F80E2E8CF0C94B1
:100A50008F070C9491070C9482030C942B05089536
:100A600024E0829FC0011124FC01E70FF11DEE0F6D
:100A7000FF1FEE0FFF1FE60FF11DEE0FFF1FE455E6
:100A8000FF4F859194910895FC01EE0FFF1FE455EF
:100A9000FD4F8591949108950E9430050E94BF06F4
:100AA000811520E4920708F08DC0811540E394077A
:100AB00008F0E8C0803E910508F071C0803C9105C7
:100AC00008F0CCC0883A910580F4853A910508F089
:100AD000CAC08130910509F46EC020F084309105C0
:100AE00008F069C090E080E008958D3B9105D0F753
:100AF000883A910509F404C1893A910509F403C1C2
:100B00008A3A910509F402C18B3A910509F401C1B1
:100B10008C3A910509F400C18B3B910509F4FFC0A3
:100B20008C3B910509F4FEC08D3A910509F4FDC096
:100B3000803B910509F4FCC08E3A910509F4FBC095
:100B40008F3A910509F4FAC0813B910509F4F9C087
:100B5000823B910509F4F8C0833B910509F4F7C085
:100B6000843B910509F4F6C0853B910509F4F5C075
:100B7000863B910509F4F4C0873B910509F4F3C065
:100B8000883B910509F4F2C0893B910509F4F1C055
:100B90008A3B910509F4F0C080E094E408958F3F0A
:100BA000910509F048F4803F910508F067C0883E40
:100BB000910508F097CF0895811520E2920708F07B
:100BC0005FC00895811543E5940760F5811522E51E
:100BD000920708F062C0811541E5940708F058C0FB
:100BE000811520E5920708F450C09C0154E0369529
:100BF00027955A95E1F7922F9370482F437021E083
:100C000030E002C0220F331F4A95E2F73C68392BCF
:100C100086958695837040E2849FC0011124822BC3
:100C2000932B0895811545E5940750F4811524E52B
:100C3000920708F446C0982F8827846F906A089519
:100C4000811546E5940708F450C09C0130569F700A
:100C50002115304108F046CF90620895805C9109DB
:100C60000E9444050895853A910509F443C0863AE7
:100C7000910509F042C082E890E4089590650895D6
:100C80009F70EECF9927906C08959F70906A089599
:100C9000982F8827816F906A0895AC01437055277B
:100CA00021E030E002C0220F331F4A95E2F786951B
:100CB000869540E2849FC0011124822B932B9C686F
:100CC0000895AC014370552721E030E002C0220FA7
:100CD000331F4A95E2F78695869540E2849FC001CE
:100CE0001124822B932B9A680895982F88278827A0
:100CF0009F71B2CF81E890E4089583E890E408956D
:100D000082EE94E4089589EE94E408958AEE94E4E2
:100D1000089585EB94E4089586EB94E4089583EBBD
:100D200094E4089584EB94E4089587EB94E40895A3
:100D30008CEC94E408958DEC94E4089583E895E4B4
:100D400008958AE895E4089582E995E4089584E990
:100D500095E4089581E296E4089583E296E4089587
:100D600084E296E4089585E296E4089586E296E4A6
:100D7000089587E296E408958AE296E41CCF8238CB
:100D8000910549F1B0F48133910509F45CC048F450
:100D90008932910509F452C08A32910509F458C08C
:100DA00008958533910509F444C08933910599F07C
:100DB0000895833E910531F138F4803E910591F01C
:100DC000823E9105B1F00895863E910511F1873E6E
:100DD000910541F1089520911B022370C9F080EE26
:100DE00090E0089520911B0220FF12C089E390E05B
:100DF000089520911B0222FF0BC024FF2EC090E01B
:100E000080E0089520911B0222FD2AC024FDF7CF27
:100E1000089520911B0223FFFBCF24FDF0CF87EE26
:100E200090E0089520911B0223FFF0CF86EE90E022
:100E3000089520911B0225FD16C0089520911B02E4
:100E400025FD14C0089520911B0226FD12C00895AF
:100E500020911B0226FD10C0089583EE90E00895B6
:100E600082EE90E0089589E290E0089585E390E0B5
:100E700008958AE290E0089581E390E0C9CF089553
:100E80000F931F93CF938C01FB018281811106C0C8
:100E9000C1E08C2FCF911F910F910895C091410116
:100EA000C11125C00531104799F70E943F0781E025
:100EB000809341010E94A9199093400180933F01C2
:100EC00010923401109236011092350110923801BF
:100ED0001092370110923A011092390110923C01A0
:100EE00010923B0110923E0110923D01D2CF8091B1
:100EF0003F01909140010E94B519883C910540F650
:100F000080913401E82FF0E0EE0FFF1FEB5CFE4F05
:100F1000118300838F5F80933401C0E0BACF0C94BB
:100F20007E030C947F03CF93DF9385B7806885BFE2
:100F300085B7806885BFA8E1B1E04CE151E0C1E030
:100F4000D0E08D91E82FE295EF70F0E061A18F7015
:100F50009E0101C0220F8A95EAF7922F9095962361
:100F600091A382A1822B82A34A175B0751F7A4E1C8
:100F7000B1E048E151E0C1E0D0E08D91E82FE29589
:100F8000EF70F0E061A18F709E0101C0220F8A9581
:100F9000EAF7922F9095962391A382A1822B82A3A8
:100FA0004A175B0751F710924601109242011092C6
:100FB000470110924301109248011092440110928F
:100FC000490110924501DF91CF910C9427056F9252
:100FD0007F928F929F92AF92BF92CF92DF92EF92C9
:100FE000FF920F931F93CF93DF93C2E4D1E008E108
:100FF00011E09CE1E92E91E0F92ECC24C394D12C90
:10100000BB24B394A8801882D8018D918D01E82F5C
:10101000E295EF70F0E091A18F70A60101C0440F3E
:101020008A95EAF7892F842B81A382A1842E80944C
:10103000882182A3B0EABA95F1F784E1682E81E0B5
:10104000782E90E080E0D3013D913D01632F6295C1
:101050006F7070E0DB0190962C9198803F70B60124
:1010600001C0660F3A95EAF7622320E031F42C2D97
:10107000082E01C0220F0A94EAF729292883019635
:101080008430910501F781A1882181A382A1482B99
:1010900042A38881A81641F0B0924A010E94A91982
:1010A00090934C0180934B012196E016F10609F0D4
:1010B000A9CF80914A018823D1F080914B01909172
:1010C0004C010E94B519069790F0809142018093DF
:1010D00046018091430180934701809144018093B0
:1010E0004801809145018093490110924A010E9474
:1010F000290581E0DF91CF911F910F91FF90EF9033
:10110000DF90CF90BF90AF909F908F907F906F9027
:101110000895E82FF0E0EA5BFE4F8081089508957E
:1011200035B1242F2095232335B1432B3FB7F894B5
:10113000FC01680F791FE617F70711F43FBF089508
:10114000819198E045B9000000C087FF25B9880F5C
:10115000000000C000C000C025B900C09A9591F7FA
:10116000EACF24B1242B24B99B01220F331F620F35
:10117000731F0E94900887EC90E00197F1F700C080
:101180000000089542E00C94B108CF92DF92EF92F4
:10119000FF920F931F93CF93DF93E901662309F426
:1011A00066C0E42EF12CEFEFF0E0E61BF109EE9DB6
:1011B0008001EF9D100DFE9D100D1124212FE12FB8
:1011C000FF27EE1AFF0A5CE3C52ED12CB6010E9460
:1011D000B725FB01BC01E69EC001E79E900DF69E7F
:1011E000900D1124B6010E94B725E230F10589F176
:1011F00068F4812F262F210F309781F0242F461B72
:10120000319761F080E020E040E008C0E430F10573
:1012100051F128F1842F861B3597A1F7E42FF0E0D8
:10122000E754FC4F4491E22FF0E0E754FC4F9491D7
:10123000E82FF0E0E754FC4FE49149839883EA8378
:10124000DF91CF911F910F91FF90EF90DF90CF90A2
:101250000895862F810FE42F412F2E2FDFCFE42F0B
:10126000E61B842FF9CF842F462F410FD7CF842F31
:10127000242FD4CF88E090E00C94ED25AB01BC0185
:1012800088E090E00C940B26ECE0F2E083E08083B1
:1012900010920D028FEF8283838360910C02709114
:1012A0000D0280910E0290910F020C943E098091E4
:1012B0000C0280FF06C061E070E084E192E00C94D3
:1012C000C208109215021092140210921602F3CF67
:1012D000E4E1F2E08183608342830C945709EF924A
:1012E000FF920F931F93CF93DF9300D01F92CDB740
:1012F000DEB7182FE92EF62E042F80910C02909164
:101300000D02A0910E02B0910F02809310029093F3
:101310001102A0931202B093130280910C0280FF7D
:101320001FC09E012F5F3F4F812F9E2D0E94C50839
:101330008091100210FB87F980931002169580911E
:1013400011028078812BE0FA87F980931102F092E4
:101350001202009313024B8169818A810E946809FD
:101360000F900F900F90DF91CF911F910F91FF90F1
:10137000EF9008950F931F93CF93DF93EC01062F07
:10138000142F90910C0290FF43C0892F8E778230EA
:1013900021F5CE010E946F0980910C02C0FB87F9F4
:1013A00080930C02C69580910D028078C82BD0FBEB
:1013B000C7F9C0930D0200930E0210930F026091C3
:1013C0000C0270910D0280910E0290910F02DF913C
:1013D000CF911F910F910C943E09892F86958F73A1
:1013E0002EE3280F2F73243018F410910F02D4CF5E
:1013F000865C8F73893080F6991F9927991FD09149
:101400000D02CD2FCC0FC92BD7FBDD27D0F9C4CFD0
:10141000DF91CF911F910F910895ECE0F2E02081D0
:10142000221F2227221F30910D02432F440F842FA9
:10143000822B37FB992790F9089668E671E00E94A5
:10144000CB25438162810C94BA0920910C02221FA2
:101450002227221F30910D02432F440F842F822B0D
:1014600037FB992790F98830910540F4805A9E4FB8
:1014700040910F0260910E020C94BA09089768E639
:1014800071E00E94CB25F4CF60910E02683F90F48A
:10149000685F80910C02881F8827881F90910D0239
:1014A000292F220F97FB992790F940910F02822B49
:1014B0000C94BA096FEFEDCF60910E02683090F096
:1014C000685080910C02881F8827881F90910D0218
:1014D000292F220F97FB992790F940910F02822B19
:1014E0000C94BA0960E0EDCF40910F02483F90F4B0
:1014F000485F80910C02881F8827881F90910D02F9
:10150000292F220F97FB992790F960910E02822BC9
:101510000C94BA094FEFEDCF40910F02483090F094
:10152000485080910C02881F8827881F90910D02D7
:10153000292F220F97FB992790F960910E02822B99
:101540000C94BA0940E0EDCF90910C0290FF3BC0A3
:101550009178811126C0926090930C0260910C02E8
:1015600070910D0280910E0290910F020E943E092F
:1015700080910C02982F9E779230D9F410926201DC
:10158000881F8827881F90910D02292F220F97FB13
:10159000992790F940910F0260910E02822B0C94D2
:1015A000BA09893110F09063D7CF8F73880F982BC9
:1015B000D3CF982F9695925C9F73963108F791E060
:1015C00090936201DDCF08958091DF018160809367
:1015D000DF0181E0809363010E940919811104C039
:1015E0000E94E8180E9444090E943A0960930C0284
:1015F00070930D0280930E0290930F026E7761F448
:101600000E9444090E943A0960930C0270930D02F3
:1016100080930E0290930F0281E08093620180918B
:101620000C0280FF04C086958F730C94A40A089561
:1016300080910C0286958F738F5F893108F081E06D
:101640000C94A40A90910C02892F8E7F90FF8160E8
:1016500080930C0260910C0270910D0280910E0239
:1016600090910F020E943E0980910C0280FF04C0FD
:1016700086958F730C94A40A109262012FEF80E775
:1016800092E0215080409040E1F700C000000C94AF
:101690005709CF93C82F80916001909161010E94FA
:1016A000B519EC2FF0E0EB54FD4FE491E817190663
:1016B00009F010F50E94A9199093610180936001CF
:1016C000E0915F01F0E0E754FD4F449180910C02FE
:1016D000881F8827881F90910D02292F220F97FBC2
:1016E000992790F960910E02822B0E946F098091D8
:1016F0005F018F5F80935F01CF910895CF93C82FD3
:1017000080915D0190915E010E94B519EC2FF0E08F
:10171000EE54FD4FE491E817190609F0E8F40E9431
:10172000A91990935E0180935D0140910F02609131
:101730000E0280915B0190915C010E946F09809183
:101740005B0190915C01019668E671E00E94B7250B
:1017500090935C0180935B01CF9108951F93CF9389
:10176000DF93182F8091590190915A010E94B51969
:10177000E12FE695F0E0EE54FD4FE491E8171906ED
:1017800009F038F50E94A91990935A0180935901E4
:101790008091570190915801C8E6D1E0BE010E94A6
:1017A000B72524E132E040910F0260910E020E94C1
:1017B000C5080E945709809157019091580110FF68
:1017C0000CC00196BE010E94B725909358018093EA
:1017D0005701DF91CF911F9108950197F6CFEF92B6
:1017E000FF920F931F93CF93DF93C82F1FEF80FFBC
:1017F00011E080915501909156010E94B519C6954E
:10180000EC2FF0E0E155FD4FE491E817190611F0D7
:1018100008F045C00E94A919909356018093550184
:10182000109215021092140210921602C7E0D0E036
:1018300000E087E0E82EF12C80915401800F87FDB5
:101840008F5F81111EC020910F022C9FC0012D9F20
:10185000900D1124B7010E94CB25462F80910C02D8
:10186000881F8827881F90910D02592F550F97FBCD
:10187000992790F924E132E060910E02852B0E94B5
:10188000C508010F2197C1F60E945709113071F464
:1018900080915401882319F0815080935401DF9185
:1018A000CF911F910F91FF90EF90089510925401E6
:1018B000F6CF1F93CF93DF9300D01F92CDB7DEB743
:1018C000182F80915201909153010E94B519E12F78
:1018D000F0E0E455FD4FE491E817190609F0D8F55A
:1018E0000E94A91990935301809352011A82198280
:1018F0001B8217E080910C02881F8827881F909117
:101900000D02592F550F97FB992790F99E012F5FD4
:101910003F4F40910F0260910E02852B0E94C50837
:10192000115041F78A8180931502898180931402B6
:101930008B81809316020E9457099091000180913B
:101940005101913099F48A3F6CF489EF80935101F1
:101950008FEF809300010F900F900F90DF91CF9148
:101960001F910895815080935101F5CF88302CF05C
:1019700087E08093510181E0ECCF8F5FF4CF8091BD
:101980004F01909150010E94B519883E934010F18B
:101990000E94A9199093500180934F0180914D01AD
:1019A00090914E0101968170992790934E018093FA
:1019B0004D0124E132E040910F0260910E0250E5AA
:1019C000FC015E9FC0015F9F900D11240E94C5081D
:1019D0000C945709089580916201882371F18091D8
:1019E0000C0286958F739EE3980F9F73943018F4C2
:1019F00082500C94490B9AE3980F9F73933018F41C
:101A000086500C947E0B97E3980F9F73963018F4D2
:101A100089500C94AE0B91E3980F9F73963018F495
:101A20008F500C94EF0B9BE2980F9F73933018F438
:101A300085510C94590C0C94BF0C08959093690136
:101A4000809368010895E0916801F09169013097F1
:101A500021F00190F081E02D099480E00895E0915B
:101A60006801F0916901309721F00280F381E02D47
:101A700009940895E0916801F0916901309721F08F
:101A80000480F581E02D099408952091660130913C
:101A900067012817390771F09093670180936601F9
:101AA000E0916801F0916901309721F00680F7819B
:101AB000E02D099408952091640130916501281763
:101AC000390771F09093650180936401E09168019A
:101AD000F0916901309721F00084F185E02D09949F
:101AE000089508950C94710D0E94A0190E94930707
:101AF0000E94691A0C94E40ABF92CF92DF92EF928F
:101B0000FF920F931F93CF93DF93CDB7DEB72A9742
:101B10000FB6F894DEBF0FBECDBF0E94E7078BE67D
:101B2000C82E81E0D82E10E000E0B02E802F0E9459
:101B30008908E82EF601F1906F01F81609F45AC0F1
:101B40008091DF0181FD0E948F0890E080E0FE24FB
:101B50002F2D30E0482FB901082E02C075956795EA
:101B60000A94E2F760FF41C08E83BF8281E090E07B
:101B70006C0102C0CC0CDD1C4A95E2F72E2D30E042
:101B80002C213D21232B09F480E088870E94A9198C
:101B90008160782F9A8789874E815F8168858A85E1
:101BA0000E94210EF801E559FE4F80818C2580832B
:101BB0000E94ED1C0E94230D90916A01891789F102
:101BC0000E94230D80936A012A960FB6F894DEBF17
:101BD0000FBECDBFDF91CF911F910F91FF90EF907E
:101BE000DF90CF90BF900C942D0501968430910525
:101BF00009F0B0CF0F5F1F4F0430110509F095CFEA
:101C00008FEF89838A831B820E94A9198160782FB4
:101C10009D838C8349815A816B818D810E94210E25
:101C2000C7CF2A960FB6F894DEBF0FBECDBFDF91A7
:101C3000CF911F910F91FF90EF90DF90CF90BF90C9
:101C40000895CF93DF93CDB7DEB72B970FB6F894F7
:101C5000DEBF0FBECDBF4F83588769877A878B87DA
:101C60001E821D8285E0FE013796DE0111960190ED
:101C70000D928A95E1F749815A816B817C818D8132
:101C80009E812B960FB6F894DEBF0FBECDBFDF91BD
:101C9000CF910C949E14882309F4D8C0823871F433
:101CA0000E94230D81FDD2C089E30E94F1170E949A
:101CB000B91889E30E942E180C94B918833859F486
:101CC0000E94230D80FDC2C083E50E94F1170E948F
:101CD000B91883E5EFCF843859F40E94230D82FDB3
:101CE000B5C087E40E94F1170E94B91887E4E2CFDB
:101CF0009CEF980F913A18F40E94F117DDCF90E213
:101D0000980F983050F4877091E001C0990F8A9530
:101D1000EAF7892F0E947018CFCF9BE5980F933078
:101D200070F4853A31F0863A39F083E890E00C940B
:101D3000450D81E890E0FBCF82E890E0F8CF98E590
:101D4000980F953108F082C0883A09F440C0893A6A
:101D500009F440C08A3A09F440C08B3A09F440C003
:101D60008C3A09F440C08B3B09F440C08C3B09F429
:101D700040C08D3A09F440C0803B09F440C08E3A1F
:101D800009F440C08F3A09F440C0813B09F440C0D7
:101D9000823B09F440C0833B09F440C0843B09F412
:101DA00040C0853B09F440C0863B09F440C0873BF6
:101DB00009F440C0883B09F440C0893B09F440C0A5
:101DC0008A3B09F440C090E080E00C945B0D82EE09
:101DD00090E0FBCF89EE90E0F8CF8AEE90E0F5CF6F
:101DE00085EB90E0F2CF86EB90E0EFCF83EB90E0D5
:101DF000ECCF84EB90E0E9CF87EB90E0E6CF8CEC82
:101E000090E0E3CF8DEC90E0E0CF83E891E0DDCF90
:101E10008AE891E0DACF82E991E0D7CF84E991E0D6
:101E2000D4CF81E292E0D1CF83E292E0CECF84E2C0
:101E300092E0CBCF85E292E0C8CF86E292E0C5CFB8
:101E400087E292E0C2CF8AE292E0BFCF0895882372
:101E500009F44BC0823871F40E94230D81FF45C004
:101E600089E30E94F1170E94B91889E30E942E1895
:101E70000C94B918833859F40E94230D80FF35C0A3
:101E800083E50E94F1170E94B91883E5EFCF8438EB
:101E900059F40E94230D82FF28C087E40E94F117A5
:101EA0000E94B91887E4E2CF9CEF980F913AF0F2C4
:101EB00090E2980F983050F4877091E001C0990F2C
:101EC0008A95EAF7892F0E947618D2CF9BE5980F62
:101ED000933020F490E080E00C94450D885A8531D1
:101EE00020F490E080E00C945B0D0895882321F0AD
:101EF0000E9470180C94B9180895882321F00E944C
:101F000076180C94B91808958F929F92AF92BF9251
:101F1000DF92EF92FF920F931F93CF93DF937C0199
:101F2000D62FC72FFC01058102950F701281111168
:101F30000E948F180E94EA17D82E882371F011236F
:101F400021F180E28D0F883000F182E00E94D417E9
:101F50000E94EA1791E0D82ED926EC2FE295EF7077
:101F6000F0E0EB54F04F0C94DF25C70FC70F1710AC
:101F7000171059107510F40FF40F8010F40F18118A
:101F800018118B11F40FF40F9411D12CE6CF0C2FF4
:101F90000F70C07F11F00295007F1123A9F000237C
:101FA00059F080E28D0F883010F0D11109C0802FD8
:101FB0000E9470180E94B9188D2F0E944B0E14C0F9
:101FC000802F0E948118F6CF8D2F0E94270F0023AB
:101FD00059F080E28D0F883010F0D11124C0802F8D
:101FE0000E9476180E94B918DD2009F4A4C10E944D
:101FF000C71780FDA0C1F70112820E94C1170E947D
:102000003D16C7010E94A7110E94C117DF91CF9111
:102010001F910F91FF90EF90DF90BF90AF909F9036
:102020008F900C945E16802F0E948718DBCFFC2FB8
:10203000FF70BF2EC07FC03219F0B29480EFB8227B
:10204000DD2369F0D13029F1112369F1002359F022
:10205000F701858180FFB0CF8F70858304C0112385
:1020600061F0011104C08B2D0E94760FBDCF8B2D26
:102070000130D1F70E94A318B7CF011106C00E940A
:10208000A6188B2D0E947D0FAFCF013009F4ACCF85
:10209000F6CF112321F0063008F0A6CFE4CF0530AB
:1020A00008F0A2CFEECF002361F38D2F0E94270FFF
:1020B0009BCF8C2F86958695837069F0813009F0CF
:1020C00093CF8D2F9C2F9370111102C090E080E070
:1020D0000E945B0D89CF8D2F9C2F9370111102C030
:1020E00090E080E00E94450D7FCF8D2F112329F0D5
:1020F0000E94F61B0E94E21C77CF0E945E1CFACF62
:102100008C2F837009F047C011116ECF2D2F2295AF
:1021100026952770220F220F6D2F6F70862E912C1F
:10212000B12CA12C022E04C0880C991CAA1CBB1C2B
:102130000A94D2F760E070E0CB01D4FF0FC06FE0EB
:1021400070E080E090E004C0660F771F881F991F41
:102150002A95D2F76095709580959095C695C6950D
:10216000C370C23051F080F4682979298A299B29EB
:10217000C13071F00E94E61537CF682979298A2984
:102180009B290E94021630CF0E94E615C501B401BA
:102190000E94CA1529CF8695112311F08C2F8170CA
:1021A000882309F421CF2D2F229526952770220F01
:1021B000220F6D2F6F70862E912CB12CA12C022E28
:1021C00004C0880C991CAA1CBB1C0A94D2F760E0BE
:1021D00070E0CB01D4FF0FC06FE070E080E090E0D2
:1021E00004C0660F771F881F991F2A95D2F7609544
:1021F000709580959095C695C695C370C23051F084
:1022000080F4682979298A299B29C13071F00E94BC
:10221000C016EACE682979298A299B290E94DC16F2
:10222000E3CE0E94C016C501B4010E94A416DCCE04
:10223000E0E2ED0FE53108F062C0F0E0EE5DFE4E49
:102240000C94DF253711371137113711371137113A
:10225000371137113711371137113711371137113E
:102260003711371144115211591160116A11DF7081
:102270008C2F8F71112321F00E943D168D2FF4CEEB
:102280000E945E168D2FFECE112341F0053008F01E
:10229000ABCE8C2F8F710E948316A6CE063008F02D
:1022A000A3CEF7CF8C2F8F71112339F00E943D16EA
:1022B0009BCE8C2F8F711123C9F30E945E1694CE92
:1022C000112329F08C2F8F710E9428168DCE0E9429
:1022D0001E168ACE112349F0CF718C2F0E943D1615
:1022E00063E08C2F0E94CB177FCE81E00E94D41731
:1022F000023008F479CE82E00E94D41775CE112303
:1023000029F0011159CE8C2F8F71D0CF0111CDCE74
:102310008C2F8F71D2CF4C2F4F706D2FC7010E9421
:102320007B030E94471560CE4C2F4F706D2FC70165
:102330000E942F0559CEDF91CF911F910F91FF90F1
:10234000EF90DF90BF90AF909F908F9008950F9384
:102350001F93CF93DF93EC01988189812B813C817E
:10236000232B39F08F3F19F481E09F3F19F080E073
:1023700001C081E080FD17C0CE010E949403882334
:1023800091F0688179818A810E949D178C010E9459
:10239000F8160E94BF15B801CE01DF91CF911F91B1
:1023A0000F910C94840FDF91CF911F910F9108959D
:1023B0000E948F180E94A0180E9462180E94B918EB
:1023C0000E948F1D0E94E21C90E080E00E94450D5B
:1023D00090E080E00C945B0D0E947E180C94D81164
:1023E0000E949317E92FE295EF70E250EE30E0F48F
:1023F000F0E0E350FE4E0C94DF250B120B1214128A
:10240000141216121412141214120B120B121B12A5
:10241000141214121B12803F19F020F4803E20F495
:1024200081E00895843FE1F380E00895803EC0F3A9
:10243000813FD1F7F5CF93FB882780F90895CF939B
:10244000DF9300D000D01F92CDB7DEB70F900F9072
:102450000F900F900F90DF91CF910895CF93DF935E
:1024600000D000D000D0CDB7DEB726960FB6F894D6
:10247000DEBF0FBECDBFDF91CF9108951F93CF93E5
:10248000DF93C091700116E0809171018C1304C03C
:10249000DF91CF911F910895D0E01C9FF0011D9F07
:1024A000F00D1124EE58FE4F4081518162817381FD
:1024B000848195810E942E122196C770E5CF4091AC
:1024C000A2015091A3016091A4017091A501809196
:1024D000A6019091A7010C942E121F93CF93DF9326
:1024E0008091A701807FD1F48091A4018823B1F06D
:1024F00080917001D0917101B091A201C091A301AE
:102500004091A5015091A601A1E0BF3F09F0A0E0D4
:10251000BA016095709516E0D81304C0DF91CF9191
:102520001F91089521E04115510521F02A2FCF3F39
:1025300009F020E090E020FD38C0189FF001199FBD
:10254000F00D1124EE58FE4F21812C132EC0208156
:102550002B132BC02281211128C023813481241701
:10256000350700F1241B350B283C3105F0F4209190
:10257000A7012F7020612093A70126E0289FF0017A
:10258000299FF00D1124E958FE4F80818F708061E2
:10259000808382EA91E00E94A711DF91CF911F9181
:1025A0000C943E12260F371FDFCF01968770B4CFF1
:1025B000AF92BF92CF92DF92EF92FF920F931F9351
:1025C000CF93DF93CDB7DEB761970FB6F894DEBF38
:1025D0000FBECDBF8C0185E0F801DE011D96019094
:1025E0000D928A95E1F7D8014C9111965C91119763
:1025F0001296EC903091A2016091A3018091A50107
:102600009091A60121E0009731F06F3F19F421E08D
:102610003F3F09F020E0B22FB170BB2E20FD80C1FA
:10262000F801C380D480A090A401AA2009F427C196
:10263000C816D906D0F1D601A81BB90BCD01FF24CD
:10264000F394883C910508F0F12C8091A701982F14
:10265000907FFF2009F4CAC0911187C0FE2C65133A
:1026600029C0341327C0E11025C08F70806180938A
:10267000A7010E945F1282EA91E00E94A711809157
:10268000A701F80185838F2D61960FB6F894DEBF00
:102690000FBECDBFDF91CF911F910F91FF90EF90B3
:1026A000DF90CF90BF90AF900895809590958C0D5E
:1026B0009D1DC5CF81E0CD2831F05F3F19F481E049
:1026C0004F3F09F080E080FD24C081E08E25F82F87
:1026D000F170DF2E80FF3FC0809170012091710169
:1026E00036E0821318C04D875E878D859E850E94D7
:1026F0009317292F22952F70223008F1243030F5BE
:102700009F7009F1D80115969C91907FE1F4FB2C04
:10271000BACF80E0DCCF90E0389FF001399FF00D18
:102720001124EE58FE4F6181561306C06081461396
:1027300003C062816E110FC001968770D2CF9F7067
:1027400011F0882321F3805E883008F3C8010E94CD
:10275000A711BD2CDCCFEE2009F495CF8091A70105
:1027600081608093A701F12C8ECF651312C03413C2
:1027700010C0E1100EC0F8018583C8010E94A711A6
:1027800086E0F801A2EAB1E001900D928A95E1F7A6
:1027900041C04D875E878D859E850E94F0118823FC
:1027A00009F4C8C0EE2009F4C5C08091A7018032A9
:1027B00070F02091A2013091A30138872F831986F0
:1027C000DB86CA868C87CE0107960E94A71186E019
:1027D000F801A2EAB1E001900D928A95E1F70E941A
:1027E0006D120E945F12FF24F3944DCF911115C01A
:1027F0007C2DD98AC88A6E2D89890E941F1282EA8F
:1028000091E00E94A71186E0E2EAF1E0DF011D926B
:102810008A95E9F70E945F1236CF651312C0341310
:1028200010C0E1100EC0F8018583C8010E94A711F5
:10283000E2EAF1E086E0DF011D928A95E9F7FA2CE1
:1028400022CF4D875E878D859E850E94F01188235B
:1028500009F470C0EE2009F46DC08091A7018032A8
:1028600008F4B5CF2091A2013091A3013A832983C6
:102870001B82DD82CC828E83CE010196A6CFC81644
:10288000D90638F1F601E81BF90BCF01F12C883C91
:10289000910508F03DC0FE2CEE2009F44BC06513F5
:1028A00026C0341324C08091A70180FD17C0982F43
:1028B000907FA1F0D80115968C931597903F09F45D
:1028C0005CCF982F907F905F8F70892B15968C939B
:1028D00054CF809590958C0D9D1DD8CF86E0F80142
:1028E000A2EAB1E001900D928A95E1F7CCCE4D8736
:1028F0005E878D859E850E94F011811168CF809141
:10290000A70181608093A701C8010E94A711BBCED7
:102910007C2DD98AC88A6E2D89890E941F1273CF97
:10292000EE2041F04D875E878D859E850E94F011D7
:1029300081114DCFC8010E94A71155CF1F93CF938E
:10294000DF93CDB7DEB72C970FB6F894DEBF0FBE7E
:10295000CDBF4F83588769877A878B879C87CE0145
:1029600007960E94D812882309F442C09F81888567
:102970002A853B85232B39F08F3F19F481E09F3F57
:1029800019F080E001C081E080FD08C04F815885CA
:1029900069857A858B859C850E942E1216E0809130
:1029A000700190917101891709F467C0819FC0017E
:1029B00011248E589E4F0E94D812882309F45DC0BE
:1029C000E09170011E9FF0011124EE58FE4F4081EE
:1029D000518162817381848195810E942E12809140
:1029E000700190E001968770992780937001D7CF8E
:1029F00086E0FE013796DE01119601900D928A95D0
:102A0000E1F79F8188852A853B85232B39F08F3F0D
:102A100019F481E09F3F19F080E001C081E080FD62
:102A2000BDCF2091710130E0C901019687709927CF
:102A3000409170014817190699F096E0929FD001D5
:102A4000939FB00D1124AE58BE4FFE0131960190F8
:102A50000D929A95E1F7809371010E943E129ECFEC
:102A60000E94EC11109271011092700186E0E2EA6E
:102A7000F1E0DF011D928A95E9F72C960FB6F894E4
:102A8000DEBF0FBECDBFDF91CF911F910895EF92B2
:102A9000FF920F931F93CF93DF938C01892B81F0CB
:102AA000F12CEE24E394E8012196F8018491843717
:102AB00070F4843008F05FC08130B1F08230A1F151
:102AC000DF91CF911F910F91FF90EF90089585377F
:102AD00009F44CC008F43DC09CE7980F903780F78C
:102AE0008F770E94270F49C00E5F1F4FFE01849110
:102AF00090E2980F983060F48770FE2D01C0FF0FB0
:102B00008A95EAF78F2F0E9492180E94B91802C086
:102B10000E944B0E8F2D815030F2EFE9FFE031978C
:102B2000F1F700C00000F7CF0E5F1F4FFE01849148
:102B300090E2980F983050F48770FE2D01C0FF0F7F
:102B40008A95EAF78F2F0E949818DFCF0E94270FEF
:102B5000E1CF0E5F1F4FFE01C491C150D8F28FE943
:102B60009FE00197F1F700C00000F7CF0E5F1F4F05
:102B7000FE01F490CFCF0E944B0E8E01CBCF089573
:102B80006093B6017093B7018093B8019093B90137
:102B90000C94D8110F931F930091B6011091B701B7
:102BA0002091B8013091B901DC01CB01802B912B30
:102BB000A22BB32B8093B6019093B701A093B801D9
:102BC000B093B9011F910F910C94D8110F931F93DB
:102BD0000091B6011091B7012091B8013091B9016F
:102BE000DC01CB0180239123A223B3238093B60180
:102BF0009093B701A093B801B093B9011F910F91C1
:102C00000C94D8110F931F930091B6011091B70146
:102C10002091B8013091B901DC01CB0180279127C7
:102C2000A227B3278093B6019093B701A093B80170
:102C3000B093B9011F910F910C94D8111092B20169
:102C40001092B3011092B4011092B5010C94D811F6
:102C500041E050E060E070E004C0440F551F661F83
:102C6000771F8A95D2F74093B2015093B3016093D6
:102C7000B4017093B5010C94D81141E050E060E0CC
:102C800070E004C0440F551F661F771F8A95D2F766
:102C90008091B2019091B301A091B401B091B501BE
:102CA000842B952BA62BB72B8093B2019093B30165
:102CB000A093B401B093B5010C94D81141E050E059
:102CC00060E070E004C0440F551F661F771F8A95AF
:102CD000D2F740955095609570958091B201909192
:102CE000B301A091B401B091B50184239523A6232B
:102CF000B7238093B2019093B301A093B401B09332
:102D0000B5010C94D81141E050E060E070E004C0DF
:102D1000440F551F661F771F8A95D2F78091B20125
:102D20009091B301A091B401B091B501842795278A
:102D3000A627B7278093B2019093B301A093B40163
:102D4000B093B5010C94D8110F931F930091B20169
:102D50001091B3012091B4013091B501DC01CB0198
:102D6000802B912BA22BB32B8093B2019093B301B4
:102D7000A093B401B093B5011F910F910C94D81199
:102D80000F931F930091B2011091B3012091B401F0
:102D90003091B501DC01CB0180239123A223B32321
:102DA0008093B2019093B301A093B401B093B501A5
:102DB0001F910F910C94D8110F931F930091B201A2
:102DC0001091B3012091B4013091B501DC01CB0128
:102DD00080279127A227B3278093B2019093B30154
:102DE000A093B401B093B5011F910F910C94D81129
:102DF0000895990F990F890F982F977071E001C06E
:102E0000770F9A95EAF786958695869525E0829FB5
:102E1000C001112450E040E0A62FB0E0FC01E40F17
:102E2000F51FE855FE4F60819D01042E02C03695C6
:102E300027950A94E2F72170219526272723262734
:102E400020834F5F5F4F4530510541F70895990F3B
:102E5000990F890F982F977086958695869525E00E
:102E6000829FA001112470E060E080E0FA01E60F8B
:102E7000F71FE855FE4F208130E0092E02C036953D
:102E800027950A94E2F721703327062E01C0220FFE
:102E90000A94EAF7822B6F5F7F4F6530710531F737
:102EA0000895BF92CF92DF92EF92FF920F931F93FC
:102EB000CF93DF938C01C090B201D090B301E0902A
:102EC000B401F090B5018091B6019091B701A09145
:102ED000B801B091B901C82AD92AEA2AFB2ACFE160
:102EE000D0E0BC2ED701C6010C2E04C0B695A79524
:102EF000979587950A94D2F780FD0EC0219788F7A1
:102F0000B12C8B2DDF91CF911F910F91FF90EF90FE
:102F1000DF90CF90BF900895B8018C2F0E944C0590
:102F2000019761F3EECFCF93DF93EC010E9451172D
:102F3000BE01DF91CF910C944C051F93CF93DF938B
:102F4000EB0190916F01992331F0CB01DF91CF918B
:102F50001F910C949317882379F0CB010E9451178D
:102F6000182F682FCE010E94F916BE01812FDF9124
:102F7000CF911F910C944C05CB010E942717182F5D
:102F8000F4CF8091BA0185958595859508958091B6
:102F9000BA018770089598E0899F90011124622BEF
:102FA0006093BA010C943D169091BA0180958923E3
:102FB0008093BA01282F277061F4282F082E000C67
:102FC000330B9217130629F08595859585950C94FA
:102FD0005E1608959091BA01977081E009F480E03F
:102FE0000895909113019923E1F090911B0297FFAE
:102FF00018C0E82FE695E695E695EF3139F1209176
:10300000010130910201E20FF32FF11D877021E0E1
:1030100030E001C0220F8A95EAF78181822B8183FB
:1030200008952091010130910201F90132969FEF3C
:1030300040E05191851751F09F3F19F4511101C0A3
:10304000942F4F5F4E31A9F79F3F09F40895290F40
:10305000311D97FD3A95F9018283089590911301EE
:103060009923F1F090911B0297FF1AC0E82FE69583
:10307000E695E695EF3129F12091010130910201A9
:10308000E20FF32FF11D282F277081E090E001C09F
:10309000880F2A95EAF78095918189238183089585
:1030A0002091010130910201F9013296205E3F4FDB
:1030B0009191891303C0DF0111971C92E217F30766
:1030C000B9F7089581E090E0E0910101F0910201EB
:1030D000E80FF91F1082019680329105A9F7089533
:1030E0009091DE01892B8093DE010895982F9095B1
:1030F0008091DE0189238093DE0108951092DE0124
:1031000008959091DD01892B8093DD010895982F1A
:1031100090958091DD0189238093DD0108951092BF
:10312000DD0108959091DC01892B8093DC010895E5
:10313000982F90958091DC0189238093DC0108957C
:103140001092DC0108958093BB0108951092BB0199
:1031500008952091010130910201F9013196205E1C
:103160003F4F80E0919191118F5FE217F307D1F704
:103170000895E0910101F09102018091DE018083C8
:10318000E0910101F091020180819091DD01892B94
:103190008083E0910101F091020180819091DC0136
:1031A000892B80839091BB01992361F0E09101010B
:1031B000F09102018081892B80830E94A9188111DE
:1031C0001092BB0180910101909102010C942F0D8E
:1031D0006DEE7EEF90E080E00E94172660E082E0D6
:1031E00090E00E94F92560E083E090E00E94F925DC
:1031F00060E084E090E00E94F92560E085E090E0E6
:103200000E94F92540E050E0BA0188E090E00C947B
:103210000B2690E080E00E94F32521E08D3E9E4F3A
:1032200009F020E0822F089582E090E00C94E525DB
:10323000682F82E090E00C94F92583E090E00C94F4
:10324000E525682F83E090E00C94F92584E090E078
:103250000C94E525682F84E090E00C94F92580918A
:103260002102843039F11092E00188E190E020E4FD
:103270000FB6F894A895809360000FBE209360006D
:1032800080E00E942D0583B7817F846083BF83B770
:10329000816083BF7894889583B78E7F83BF0FB694
:1032A000F894A895809160008861809360001092E6
:1032B00060000FBE089508950895CF930E945B1992
:1032C0000E94E7070E945C19C0E08C2F0E948908C9
:1032D000811105C0CF5FC430C1F7CF91089581E05F
:1032E000FCCF0E94EC110E94230D0C942D051F921F
:1032F0000F920FB60F9211248F939F93AF93BF93AA
:103300008091E001811113C0809117029091180201
:10331000A0911902B0911A024196A11DB11D80938E
:10332000170290931802A0931902B0931A02BF914A
:10333000AF919F918F910F900FBE0F901F90189596
:1033400082E084BD93E095BD9AEF97BD80936E00B7
:1033500008952FB7F8948091170290911802A091C8
:103360001902B0911A022FBF0895CF92DF92EF9207
:10337000FF920F931F932FB7F8944091170250912B
:1033800018026091190270911A022FBF6A017B0125
:10339000EE24FF248C0130E020E0C016D106E206C6
:1033A000F30650F0481B590BCA011F910F91FF9073
:1033B000EF90DF90CF90089541505109F3CF1F92C5
:1033C0000F920FB60F9211248F939F93AF93BF93D9
:1033D0008091170290911802A0911902B0911A02DF
:1033E0000196A11DB11D8093170290931802A0931E
:1033F0001902B0931A02BF91AF919F918F910F90D4
:103400000FBE0F901F9018950E948B21F8942FEFFC
:1034100087EA91E6215080409040E1F700C000002B
:1034200087E090EBDC0180932A0290932B02A0931B
:103430002C02B0932D0288E19CE00FB6F894A89579
:10344000809360000FBE90936000FFCFCF92DF9219
:10345000EF92FF920F931F93CF93C0E0E82EF12CD1
:103460008C2F0E94890810E000E0C82ED12CC601E4
:10347000002E02C0959587950A94E2F780FD11C051
:103480000F5F1F4F0430110591F7CF5FC43041F734
:1034900080E0CF911F910F91FF90EF90DF90CF9040
:1034A0000895602F7C2F80E00E943005E816F90611
:1034B00039F781E0EECFCF93C82F8CE20E94261A15
:1034C000882321F08C2FCF910C94261A80E0CF9185
:1034D0000895CF930E940919811102C00E94E81833
:1034E000C5E6C15009F0D1C089E20E945B1A811182
:1034F000F8C08AE20E945B1A81110E94E81885E0F8
:103500000E945B1A81110E94041A0E941419809370
:10351000DF0187E00E945B1A882371F08BE10E9433
:103520005B1A882309F4BAC09091DF01892F8D7F3F
:1035300091FF82608093DF018091DF010E94181962
:103540000E94261990E090931C0280931B0280EE4B
:103550000E945B1A882341F090911B02892F8E7F75
:1035600090FF816080931B0289E30E945B1A88238D
:1035700041F090911B02892F8D7F91FF8260809393
:103580001B0282EE0E945B1A882341F090911B027D
:10359000892F8B7F92FF846080931B0286EE0E94AE
:1035A0005B1A882341F090911B02892F877F93FF3C
:1035B000886080931B0283EE0E945B1A882341F08F
:1035C00090911B02892F8F7E94FF806180931B0254
:1035D00085E30E945B1A882341F090911B02892F9A
:1035E0008F7D95FF806280931B0281E30E945B1AAE
:1035F000882341F090911B02892F8F7B96FF806476
:1036000080931B0281E10E945B1A882341F0909114
:103610001B02892F97FB87F9805880931B028091AA
:103620001B020E942A1987E20E945B1AC82F8EE1B2
:103630000E945B1A8111C2608FE10E945B1A8111A6
:10364000C46080E20E945B1A8111C86081E20E941E
:103650005B1A8111C06182E20E945B1A8111C06213
:1036600083E20E945B1A8111C06484E20E945B1AAB
:10367000882389F1C0688C2F0E9421196C2F70E07B
:1036800090E080E0CF910C94C0150E94E7078FE393
:103690009CE90197F1F700C0000023CF8EE00E9463
:1036A0005B1A882339F09091DF01892F8B7F92FF7D
:1036B000846040CF80E10E945B1A9091DF018823F3
:1036C00029F0892F877F93FF886034CF892F8E7FE1
:1036D00090FF81602FCFC111CECF0E941D19682F9E
:1036E000CECFCF9108958091E30180FF12C0609109
:1036F000060185E0689FB001112475956795759561
:10370000679560387105A8F561157105A1F1862FDF
:10371000089581FF09C06091060185E0689FB001AE
:10372000112475956795EDCF82FF07C06091060162
:1037300085E0689FB0011124E4CF2091E4012223A9
:10374000A9F0909105016091060185E0689FB001A4
:1037500011242917B0F6269FA001279F500D112490
:10376000692F70E0CA010E94CB25CBCF65E070E0E5
:10377000CECF8FE7089581E008958091E30180FF27
:103780000CC06091040170E075956795759567951B
:103790006115710549F1862F089581FF06C060917A
:1037A000040170E075956795F3CF6091040182FD87
:1037B0000BC09091E4019923A1F0609103018091E5
:1037C0000401961738F0682F70E06038710500F337
:1037D0008FE70895899FC001112470E00E94CB25D6
:1037E000F4CF61E070E0D7CF81E00895803F31F4FD
:1037F0000E94731B81958093E7010895813F19F41E
:103800000E94731BF8CF823F31F40E94731B819595
:103810008093E6010895833F19F40E94731BF8CF4B
:10382000893F29F40E94BD1B8093E80108958A3FD7
:1038300021F40E94BD1B8195F7CF8B3F31F40E948C
:10384000BD1B81958093E90108958C3F19F40E9476
:10385000BD1BF8CF843F31F48091E50181608093F6
:10386000E5010895853F21F48091E5018260F7CF5D
:10387000863F21F48091E5018460F1CF873F21F4F8
:103880008091E5018860EBCF883F21F48091E501CC
:103890008061E5CF8D3F31F48091E30181608093B9
:1038A000E30108958E3F21F48091E3018260F7CF18
:1038B0008F3FB9F78091E3018460F1CF803FC1F47D
:1038C0008091E70187FD1092E7018091E601811167
:1038D0000EC08091E70181110AC08091E801811139
:1038E00006C08091E901811102C01092E40108959F
:1038F000813F29F48091E70118162CF3E6CF9091CF
:10390000E601823F29F497FFE0CF1092E601DDCF78
:10391000833F19F41916CCF3D8CF893F39F480913D
:10392000E801181694F61092E801CFCF8A3F29F4E7
:103930008091E80187FFC9CFF6CF8B3F39F48091A2
:10394000E90187FFC2CF1092E901BFCF8C3F29F474
:103950008091E9011816BCF3B8CF843F31F480910F
:10396000E5018E7F8093E501B0CF853F21F4809102
:10397000E5018D7FF7CF863F21F48091E5018B7FB4
:10398000F1CF873F21F48091E501877FEBCF883F1E
:1039900021F48091E5018F7EE5CF8D3F31F4809158
:1039A000E3018E7F8093E30190CF8E3F21F48091DD
:1039B000E3018D7FF7CF8F3F09F087CF8091E3013F
:1039C0008B7FF0CF85EE91E00E943A0D0E94A919FD
:1039D0009093E2018093E10108951F93CF93DF93C9
:1039E0008091E1019091E2010E94B519AC019091A2
:1039F000E4012091070130E0911106C020910801F7
:103A00008AE0289F900111244217530780F080918B
:103A1000E601C091E7011091E801D091E90181111F
:103A20000AC0C11178C0111176C0D11174C0DF91E4
:103A3000CF911F9108959F3F19F09F5F9093E401EC
:103A4000181624F40E94731B8093E6018091E6010E
:103A500087FF05C00E94731B81958093E6011C16A9
:103A600024F40E94731B8093E7018091E70187FF94
:103A700005C00E94731B81958093E7016091E60168
:103A8000662331F1C091E701CC2311F1062E000C21
:103A9000770B880B990B0E94BE2423E333E343E3A7
:103AA0005FE30E9422250E9486246093E6016C2F2A
:103AB000CC0F770B880B990B0E94BE2423E333E3D2
:103AC00043E35FE30E9422250E9486246093E7017E
:103AD000111624F40E94BD1B8093E8018091E80137
:103AE00087FF05C00E94BD1B81958093E8011D16CC
:103AF00024F40E94BD1B8093E9018091E90187FFB6
:103B000005C00E94BD1B81958093E901DF91CF9193
:103B10001F910C94E21C9F3F09F08FCFA0CF85E04E
:103B2000E5EEF1E0DF011D928A95E9F71092E401DC
:103B30001092E301089580910A020895CF93DF93D4
:103B400000D01F92CDB7DEB79C0180912102843056
:103B500019F593E099833B832A839093E9008FEFD3
:103B60009091E800815095FD06C095ED9A95F1F78A
:103B700000008111F5CF8091E80085FF0DC050E075
:103B800040E063E070E0CE0101960E94FB1F80914F
:103B9000E8008E778093E8000F900F900F90DF91F0
:103BA000CF910895CF93DF9300D01F92CDB7DEB7AA
:103BB00020912102243031F522E029838058910997
:103BC0009B838A8383E08093E9008FEF9091E800E4
:103BD000815095FD06C095ED9A95F1F70000811191
:103BE000F5CF8091E80085FF0DC050E040E063E034
:103BF00070E0CE0101960E94FB1F8091E8008E7755
:103C00008093E8000F900F900F90DF91CF9108956F
:103C10009C01809121028430F9F482E08093E900D4
:103C20009FEF8091E800915085FD06C085ED8A9553
:103C3000F1F700009111F5CF8091E80085FF0CC0ED
:103C400050E040E065E070E0C9010E94FB1F8091F8
:103C5000E8008E778093E8000895CF93DF93EC011E
:103C6000809121028430F1F4909113019923E9F0BD
:103C700090911B0297FF19C08093E9008FEF9091FC
:103C8000E800815095FD06C095E19A95F1F7000096
:103C90008111F5CF8091E80050E040E060E270E0F3
:103CA00085FD1AC0DF91CF91089581E08093E900EE
:103CB0008FEF9091E800815095FD06C095ED9A95A3
:103CC000F1F700008111F5CF8091E80085FFEACF80
:103CD00050E040E068E070E0CE010E94FB1F809160
:103CE000E8008E778093E80080E2FE01AAEEB1E062
:103CF00001900D928A95E1F7D5CF80912002811134
:103D000009C00E948B210E94E8218091E20084601A
:103D10008093E20008951092200208950895089576
:103D20000C94711942E061EC81E00E94092142E0AB
:103D300061EC82E00E94092142E061EC83E00E9494
:103D4000092142E261EC84E00C9409218091230274
:103D5000833009F455C030F4813071F1823009F4B8
:103D600091C008958A3009F47DC08B3009F463C096
:103D7000893009F044C080912202813209F03FC0AD
:103D80008091260290912702009711F00397B9F5D0
:103D90008091E800877F8093E8008091E80082FFAF
:103DA0002AC08091F10080930A028091E8008B770D
:103DB0008093E8000C943D2180912202813AF9F42D
:103DC0008091E800877F8093E8008091260290919F
:103DD0002702892B61F460E28AEE91E070E00E9494
:103DE0004A208091E8008B778093E800089560E096
:103DF00090E080E0F3CF809121028111CECF089531
:103E000080912202813AD9F780912602909127026F
:103E1000892BA9F78091E800877F8093E800809143
:103E2000E80080FFFCCF809113018093F100809126
:103E3000E8008E77BDCF80912202813201F7809118
:103E4000260290912702892BD1F68091E800877F86
:103E50008093E8000E943D21809124028093130109
:103E60000C94EC1180912202813249F68091E80095
:103E7000877F8093E8000E943D21809125028093F6
:103E80000B02089580912202813A09F0B8CF809107
:103E9000E800877F8093E8008091E80080FFFCCFF6
:103EA00080910B02C2CF84B7877F84BF0FB6F8948E
:103EB000A8958091600088618093600010926000F6
:103EC0000FBE80E880936100109261000E94720D25
:103ED0000E948B210E94E8218091E20084608093FF
:103EE000E20078940E946A240E94740D89E091E0B7
:103EF0000E941E0D80912102853029F00E947C0DC8
:103F00000E94EB0CF7CF0E942F1980911F0288238B
:103F100089F30E945D19882369F30E94E51FEACFA7
:103F2000292F33272330310579F158F42130310519
:103F3000F1F02230310519F190E080E030E020E02E
:103F40001AC02132310599F122323105A9F76430C6
:103F500098F770E0FB01EE0FFF1FE05EFE4F20813F
:103F60003181645E7E4FFB01808190E004C082E17C
:103F700090E026E535E0FA013183208308958DE64F
:103F800090E029EE34E0F7CF99278130910561F078
:103F900028F0029789F6E9EBF4E002C0E5EEF4E0E0
:103FA000849190E09F01E7CFEDECF4E0F9CF64302D
:103FB00008F0C2CFE62FF0E0EE0FFF1FE85DFE4FE6
:103FC0002081318189E090E0D6CF80E189BD82E116
:103FD00089BD09B400FEFDCF8091D8008F7D80930C
:103FE000D8008091E00082608093E0008091E00042
:103FF00081FDFCCF0895AF92BF92CF92DF92FF92E6
:104000000F931F93CF93DF936C01EB018A010E9402
:104010005C21F82E811123C00115110539F0F8013A
:1040200080819181C81BD90BC80ED91EB12CA12C3F
:104030002097A9F08091E80085FD22C08091E800DA
:104040008E778093E80001151105A1F0F8018081B9
:104050009181A80EB91EB182A08285E0F82E8F2D25
:10406000DF91CF911F910F91FF90DF90CF90BF9084
:10407000AF9008950E945C218823D1F2F82EEFCFF3
:10408000F60181916F018093F1002197FFEFAF1A44
:10409000BF0ACECFFC018091280290912902861799
:1040A0009707A0F06115710529F49091E8009E77BB
:1040B0009093E80090E06115710551F4911108C0EA
:1040C0008091E80082FF35C080E00895BC01F2CF06
:1040D000809121028823C9F18530C9F18091E800DF
:1040E00083FD31C08091E80082FDEACF8091E80035
:1040F00080FFE1CF2091F3008091F200322F282F32
:104100006115710519F02830310558F091E028301B
:10411000310509F090E02091E8002E772093E80027
:10412000CACF81918093F100615071092F5F3F4F99
:10413000E7CF80912102882341F0853041F08091C2
:10414000E80083FFBDCF81E0089582E0089583E019
:104150000895FC0180912802909129028617970703
:10416000A0F06115710529F48091E8008E778093A5
:10417000E80090E06115710551F4911108C080913B
:10418000E80082FF36C080E00895BC01F2CF809144
:1041900021028823D1F18530D1F18091E80083FD9F
:1041A00032C08091E80082FDEACF8091E80080FF74
:1041B000E1CF2091F3008091F200322F282F61157A
:1041C000710519F02830310558F091E0283031059B
:1041D00009F090E08091E8008E778093E800CACFE4
:1041E00084918093F1003196615071092F5F3F4FA8
:1041F000E6CF80912102882341F0853041F0809103
:10420000E80083FFBCCF81E0089582E0089583E059
:104210000895982F973028F08F708093E90081E0FF
:1042200008959093E900242F762F50E0981731F0ED
:104230007091EC002091ED005091F00021FD02C042
:104240009F5FE8CF3091EB003E7F3093EB003091E1
:10425000ED003D7F3093ED003091EB003160309305
:10426000EB007093EC002093ED005093F000209150
:10427000EE0027FDE5CF80E008958091220287FFC0
:1042800013C08091E80082FF06C08091E8008B7720
:104290008093E80004C0809121028111F2CF08953B
:1042A000809121028823D9F38091E80080FFF8CF24
:1042B0008091E8008E77ECCF2091E4003091E5000A
:1042C00085E69091EC0090FF06C09091E80090FF89
:1042D00006C080E008959091E80092FDFACF909199
:1042E0002102992391F0953091F09091EB0095FD8A
:1042F00010C04091E4005091E5002417350709F300
:1043000081509A01F1F684E0089582E0089583E0F7
:10431000089581E008950E94F9210E940122E0EEB3
:10432000F0E0808181608083E8EDF0E080818F772C
:10433000808319BCA7EDB0E08C918E7F8C93808137
:104340008F7E80831092200208950F931F93CF9346
:10435000DF930E94F9210E940122C8EDD0E08881FC
:104360008F77888388818068888388818F7D888320
:1043700019BC1092210210921D0210921F0210927D
:104380001E0200EE10E0F80180818B7F808388811F
:104390008160888342E060E080E00E940921E1EED4
:1043A000F0E080818E7F8083E2EEF0E080818160AA
:1043B0008083808188608083F80180818E7F808304
:1043C000888180618883DF91CF911F910F9108953B
:1043D000E8EDF0E080818F7E8083E7EDF0E0808182
:1043E0008160808384E082BF81E0809320020C940E
:1043F000A521E8EDF0E080818E7F80831092E200BD
:1044000008951092DA001092E10008951F920F9221
:104410000FB60F9211242F933F934F935F936F9397
:104420007F938F939F93AF93BF93EF93FF9380916D
:10443000E10082FF0BC08091E20082FF07C0809103
:10444000E1008B7F8093E1000E9469248091DA0073
:1044500080FF19C08091D80080FF15C08091DA00DC
:104460008E7F8093DA008091D90080FF94C080E134
:1044700089BD82E189BD09B400FEFDCF81E0809352
:1044800021020E947D1E8091E10080FF19C0809171
:10449000E20080FF15C08091E2008E7F8093E200F1
:1044A0008091E20080618093E2008091D800806278
:1044B0008093D80019BC85E0809321020E948F1E52
:1044C0008091E10084FF29C08091E20084FF25C033
:1044D00080E189BD82E189BD09B400FEFDCF8091F4
:1044E000D8008F7D8093D8008091E1008F7E8093EB
:1044F000E1008091E2008F7E8093E2008091E200F3
:1045000081608093E20080911D02882309F449C0F4
:1045100084E0809321020E94901E8091E10083FF3D
:1045200029C08091E20083FF25C08091E100877F50
:104530008093E10082E08093210210921D0280911D
:10454000E1008E7F8093E1008091E2008E7F809376
:10455000E2008091E20080618093E20042E060E04E
:1045600080E00E9409218091F00088608093F00033
:104570000E948E1EFF91EF91BF91AF919F918F91FD
:104580007F916F915F914F913F912F910F900FBE4F
:104590000F901F90189519BC109221020E948B1E3B
:1045A00072CF8091E30087FD02C081E0B2CF83E04B
:1045B000B0CF1F920F920FB60F9211242F933F93FB
:1045C0004F935F936F937F938F939F93AF93BF931B
:1045D000CF93EF93FF93C091E900CF708091EC00EF
:1045E0001092E9008091F000877F8093F00078942A
:1045F0000E9415231092E9008091F000886080935A
:10460000F000C093E900FF91EF91CF91BF91AF917E
:104610009F918F917F916F915F914F913F912F91DA
:104620000F900FBE0F901F9018951F93CF93DF939D
:10463000CDB7DEB7AA970FB6F894DEBF0FBECDBFD9
:10464000E2E2F2E08091F100819322E0EA32F207A7
:10465000C9F70E94A61E8091E80083FF42C08091A6
:104660002202909123029A3008F03BC0E92FF0E03B
:10467000E45CFC4D0C94DF2546236A2371236A23F6
:104680007123C523E72371233C244924803879F022
:10469000823839F5809126028F708093E9008091ED
:1046A000EB0085FB882780F91092E90006C0809115
:1046B0001E0290911F02911182609091E800977FF5
:1046C0009093E8008093F1001092F1008091E8004F
:1046D0008E772DC0282F2D7F21F48823D1F08230B2
:1046E00059F18091E80083FF0AC08091E800877F3C
:1046F0008093E8008091EB0080628093EB00AA96A3
:104700000FB6F894DEBF0FBECDBFDF91CF911F91E2
:10471000089580912402813021F7933009F080E0E0
:1047200080931F021092E9008091E800877F8093B8
:10473000E8000E943D21D5CF809124028111F2CF63
:10474000809126028F7069F28093E9002091EB003E
:1047500020FFE8CF933031F48091EB0080628093AA
:10476000EB00E0CF9091EB0090619093EB0021E0A3
:1047700030E001C0220F8A95EAF72093EA001092F8
:10478000EA008091EB008860EACF8111AACF1091F6
:1047900024021F778091E3008078812B8093E300CF
:1047A0008091E800877F8093E8000E943D218091FE
:1047B000E80080FFFCCF8091E30080688093E300F5
:1047C00083E0111101C082E0809321028ACF8058DA
:1047D000823008F086CF80912402909125028C3D92
:1047E00023E09207A1F583E08A838AE289834FB7A9
:1047F000F894DE01139620E03EE051E2E32FF0E072
:1048000050935700E49120FF03C0E295EF703F5FA3
:10481000EF708E2F90E0EA30C0F0C7968D939D9395
:104820002F5F243159F74FBF8091E800877F809335
:10483000E8006AE270E0CE0101960E944A20809171
:10484000E8008B778093E8004CCFC096E7CFAE01AD
:104850004F5F5F4F609126020E94901FBC01892B21
:1048600009F43FCF9091E800977F9093E800898109
:104870009A810E94A920E3CF803809F032CF80913D
:10488000E800877F8093E80080911D028093F1000B
:104890001DCF811126CF90912402923008F021CFB4
:1048A0008091E800877F8093E80090931D020E942A
:1048B0003D2180911D02882331F084E08093210204
:1048C0000E94921E0ECF8091E30087FDF6CF81E01B
:1048D000F5CF0895CF9380912102882399F0C0915C
:1048E000E900CF708091EC0080FD0EC080E0C82B05
:1048F0001092E9008091E80083FD0E941523CF709B
:10490000C093E900CF91089580E8F1CF0E948D24F3
:104910006894B1110C941C2508950E94012588F01B
:104920009F5798F0B92F9927B751B0F0E1F0660F73
:10493000771F881F991F1AF0BA95C9F714C0B130B4
:1049400091F00E941B25B1E008950C941B25672F60
:10495000782F8827B85F39F0B93FCCF386957795E3
:104960006795B395D9F73EF49095809570956195CC
:104970007F4F8F4F9F4F0895E89409C097FB3EF4F7
:1049800090958095709561957F4F8F4F9F4F99239C
:10499000A9F0F92F96E9BB279395F695879577951A
:1049A0006795B795F111F8CFFAF4BB0F11F460FFDA
:1049B0001BC06F5F7F4F8F4F9F4F16C0882311F032
:1049C00096E911C0772321F09EE8872F762F05C046
:1049D000662371F096E8862F70E060E02AF09A95E1
:1049E000660F771F881FDAF7880F9695879597F9D6
:1049F000089557FD9058440F551F59F05F3F71F0CF
:104A00004795880F97FB991F61F09F3F79F0879535
:104A10000895121613061406551FF2CF4695F1DFBE
:104A200008C0161617061806991FF1CF869571054E
:104A3000610508940895E894BB2766277727CB0182
:104A400097F908950E9435250C94A6250E94982573
:104A500038F00E949F2520F0952311F00C948F25AB
:104A60000C94952511240C941C250E94F92470F3B4
:104A7000959FC1F3950F50E0551F629FF001729F03
:104A8000BB27F00DB11D639FAA27F00DB11DAA1F12
:104A9000649F6627B00DA11D661F829F2227B00D5F
:104AA000A11D621F739FB00DA11D621F839FA00DEA
:104AB000611D221F749F3327A00D611D231F849F3A
:104AC000600D211D822F762F6A2F11249F57504091
:104AD0009AF0F1F088234AF0EE0FFF1FBB1F661F0C
:104AE000771F881F91505040A9F79E3F510580F0D5
:104AF0000C948F250C941C255F3FE4F3983ED4F36F
:104B0000869577956795B795F795E7959F5FC1F778
:104B1000FE2B880F911D9695879597F9089597F923
:104B20009F6780E870E060E008959FEF80EC089553
:104B300000240A941616170618060906089500247C
:104B40000A9412161306140605060895092E0394F6
:104B5000000C11F4882352F0BB0F40F4BF2B11F46A
:104B600060FF04C06F5F7F4F8F4F9F4F0895AA1B58
:104B7000BB1B51E107C0AA1FBB1FA617B70710F048
:104B8000A61BB70B881F991F5A95A9F7809590957A
:104B9000BC01CD01089597FB072E16F4009407D0B1
:104BA00077FD09D00E94B72507FC05D03EF490950B
:104BB00081959F4F0895709561957F4F0895EE0FF1
:104BC000FF1F0590F491E02D0994F999FECF92BD55
:104BD00081BDF89A992780B50895A6E1B0E044E038
:104BE00050E00C941F26A8E1B0E042E050E00C94A5
:104BF0001F26262FF999FECF92BD81BDF89A019705
:104C000000B4021639F01FBA20BD0FB6F894FA9A14
:104C1000F99A0FBE08950396272F0E94FA250E9445
:104C2000F925252F0E94FA25242F0C94FA250196A8
:104C3000272F0E94FA250C94F925DC01CB01FC01F9
:104C4000F999FECF06C0F2BDE1BDF89A319600B4E5
:0E4C50000D9241505040B8F70895F894FFCFF0
:104C5E00FFBC012808140A321E9B1D2D1E081ED2F1
:104C6E001D9E1D0191909466F4F5F6F7404D363970
:104C7E002406D705A1056805FB0414052D05460578
:00000001FF
